:020000040800F2
:100000000005002021050008491400084D140008CF
:10001000A11400084D1400087514000823050008F9
:10002000230500082305000823050008F936000809
:100030002305000823050008230500082305000800
:1000400023050008230500082305000823050008F0
:100050002305000823050008E53B0008113C0008C3
:100060003D3C0008693C0008953C00082305000859
:1000700023050008230500082305000823050008C0
:10008000230500082305000823050008C9250008EA
:100090003526000889260008DD260008C13C000836
:1000A0002305000823050008230500082305000890
:1000B000F53900082305000823050008230500087A
:1000C0002305000823050008230500082305000870
:1000D000230500089D2A0008B12A0008230500080E
:1000E000293D000823050008230500082305000812
:1000F0002305000823050008230500082305000840
:10010000230500082305000823050008230500082F
:10011000230500082305000823050008230500081F
:10012000230500082305000823050008230500080F
:1001300023050008230500082305000823050008FF
:1001400023050008230500082305000823050008EF
:1001500023050008230500082305000823050008DF
:1001600023050008230500082305000823050008CF
:1001700023050008230500082305000823050008BF
:1001800023050008230500082305000823050008AF
:10019000230500082305000823050008230500089F
:1001A000230500082305000823050008230500088F
:1001B000230500082305000823050008230500087F
:1001C000230500082305000823050008230500086F
:1001D000230500082305000823050008230500085F
:1001E000D0400B1CD1409C46203AD3401843524289
:1001F00063469340184370479140031C90409C46CF
:10020000203A9340194352426346D3401943704702
:1002100053B94AB9002908BF00281CBF4FF0FF316D
:100220004FF0FF3000F07AB9ADF1080C6DE904CE63
:1002300000F006F8DDF804E0DDE9022304B07047C1
:100240002DE9F0478C460D460446089E002B51D1FF
:100250008A4217466DD9B2FA82FEBEF1000F0BD06A
:10026000CEF1200C01FA0EF520FA0CFC02FA0EF782
:100270004CEA050C00FA0EF44FEA174A250CBCFBB9
:10028000FAF81FFA87F90AFB18CC45EA0C4508FB77
:1002900009F3AB420AD9ED1908F1FF3280F023814E
:1002A000AB4240F22081A8F102083D44ED1AA4B20D
:1002B000B5FBFAF00AFB105544EA054400FB09F9C6
:1002C000A14509D9E41900F1FF3380F00A81A14565
:1002D00040F2078102383C44A4EB090440EA08409C
:1002E0000021002E61D024FA0EF4002334607360E4
:1002F000BDE8F0878B4207D9002E54D0002186E854
:1003000021000846BDE8F087B3FA83F1002940F0E8
:100310008E80AB4202D3824200F2FA80841A65EBEF
:1003200003050120AC46002E3FD086E81010BDE842
:10033000F08712B90127B7FBF2F7B7FA87FEBEF1D3
:10034000000F34D1EB1B3A0C1FFA87FC0121B3FBE1
:10035000F2F8250C02FB183345EA03450CFB08F3C1
:10036000AB4207D9ED1908F1FF3002D2AB4200F2DF
:10037000D1808046ED1AA3B2B5FBF2F002FB105516
:1003800043EA05440CFB00FCA44507D9E41900F13D
:10039000FF3302D2A44500F2B8801846A4EB0C0447
:1003A00040EA08409DE731463046BDE8F087CEF18F
:1003B000200405FA0EF307FA0EF720FA04F83A0CB7
:1003C00025FA04F448EA0308B4FBF2F14FEA1845B1
:1003D00002FB11441FFA87FC45EA044501FB0CF3BC
:1003E000AB4200FA0EF409D9ED1901F1FF3080F0AB
:1003F0008A80AB4240F2878002393D44EB1A1FFAF3
:1004000088F5B3FBF2F002FB103345EA034500FB2D
:100410000CF3AB4207D9ED1900F1FF386FD2AB42B4
:100420006DD902383D44EB1A40EA01418FE7C1F132
:10043000200722FA07F88B4005FA01F448EA030383
:1004400020FA07FE4FEA134CFD404EEA040EB5FBBE
:10045000FCF94FEA1E440CFB19551FFA83F844EAD5
:10046000054509FB08F4AC4202FA01F200FA01FA70
:1004700008D9ED1809F1FF3043D2AC4241D9A9F1B6
:1004800002091D442D1B1FFA8EFEB5FBFCF00CFB70
:1004900010554EEA054400FB08F8A04507D9E418BA
:1004A00000F1FF3529D2A04527D902381C4440EA83
:1004B0000940A4EB0804A0FB02894C45C6464D4602
:1004C00015D312D056B1BAEB0E0364EB050404FA4F
:1004D00007F7CB401F43CC40376074600021BDE874
:1004E000F0871846F8E69046E0E6C245EAD2B8EB57
:1004F000020E69EB03050138E4E72846D7E74046DA
:1005000091E78146BEE7014678E702383C4445E77B
:10051000084608E7A8F102083D442BE7704700BFF2
:1005200002E000F000F8FEE772B6394880F3088870
:10053000384880F3098838484EF60851CEF2000159
:10054000086040F20000CCF200004EF63471CEF2AA
:1005500000010860BFF34F8FBFF36F8F40F20000C0
:10056000C0F2F0004EF68851CEF200010860BFF3F1
:100570004F8FBFF36F8F4FF00000E1EE100A4EF681
:100580003C71CEF200010860062080F31488BFF3AE
:100590006F8F03F0EFF803F0CDF94FF055301F499E
:1005A0001B4A91423CBF41F8040BFAE71C49194A27
:1005B00091423CBF41F8040BFAE71A491A4A1B4B17
:1005C0009A423EBF51F8040B42F8040BF8E70020B2
:1005D0001749184A91423CBF41F8040BFAE703F06F
:1005E000CDF803F0FBF9144C144DAC4203DA54F887
:1005F000041B8847F9E700F03FF8114C114DAC425D
:1006000003DA54F8041B8847F9E703F0B5B8000093
:100610000005002000250020000000080001002047
:1006200000050020C0450008002500207825002096
:1006300078250020AC420020E0010008E00100081D
:10064000E0010008E00100082DE9F04F2DED108ACF
:10065000C1F80CD0C3689D46BDEC108ABDE8F08F90
:10066000002383F311882846A047002002F092FD62
:1006700002F038FD00DFFEE7384B6FF016022DE97F
:10068000F0411A70032200245A7007229C70DC701B
:100690001C715C719C71DC711C725C729A72DC72F0
:1006A00002F0D4FF074603F021F80546002839D1AF
:1006B0002B4B9F4238D001339F4238D0294B27F033
:1006C000FF029A4237D1F8B200F052FAA84642F23D
:1006D000107400F083FC00F051FA064678B384BB36
:1006E000464635B1204B9F4203D002F0F7FF00246D
:1006F0002646002002F0B4FF1C4B1B691B0723D4C5
:100700000EB100F035F800F08BFC00F023FE00F095
:10071000DBFE0546D4B900F0D7FC4FF47A7002F046
:100720003FFDF7E78046D4E780460446D1E704461C
:100730004FF00108CDE780464FF47A74C9E70446CC
:10074000CFE74FF47A74CCE70024DCE700F0BCFE7E
:10075000401BA042DFD900F00BF8D8E77825002035
:10076000010007B0000008B0263A09B000040240BA
:1007700010B51E4B1E4953F8042F013200D110BD95
:100780008B42F8D11B4C1C4B22689A422CD91B4B34
:100790009B6803F1006303F580339A4224D202F090
:1007A00071FF02F083FF002000F0EEFD144B0220E9
:1007B000187000F01DFE134B1A6C00221A64196E9B
:1007C0001A66196E596C5A64596E5A665B6E72B627
:1007D0000D4A0E4B13601B682268202181F311889B
:1007E0009D4683F30888104710BD00BFFCFF00083A
:1007F0001C00010804000108FFFF00087825002004
:10080000842500200038024008ED00E000000108C7
:1008100009490B6849F269009AB21B0C00FB0233CC
:10082000064A0B60136844F2506198B21B0C01FB3E
:100830000030106080B27047102500200C25002089
:1008400010B500211022044600F0EEFD034B03CB4F
:10085000206061601868A06010BD00BF107AFF1FA3
:10086000F0B51F4CBBB000F02FFEA368C31AF92BE4
:1008700030D906AD2346A06028220021284601F089
:10088000B1FB04F10E0000F0C7FD0023C6B2591DF4
:100890005F1CDBB2B3424FEAC10107DA0E332344D7
:1008A0000822284601F09EFB3B46F0E70123039314
:1008B0000823207B02930B4B0193C1F3CF0130231C
:1008C000059100930146049503A3D3E9002306484C
:1008D00001F058F93BB0F0BD78F6339F93CACD8D47
:1008E000C8350020D5350020A035002070B50D4654
:1008F00014461E4601F0ECF850B9022E0ED1012C20
:100900000CD112A3D3E90023C5E90023012070BD57
:10091000052C14D003D8012C09D0002070BD282C40
:1009200009D0302CF9D10BA3D3E90023ECE70BA3BA
:10093000D3E90023E8E70BA3D3E90023E4E70BA303
:10094000D3E90023E0E700BFAFF30080401DA12002
:1009500026812A0B78F6339F93CACD8D9E6AC421D7
:10096000818A46EE26417272DF25D7B7F017304AEA
:1009700039059E5638B504460D46034620222846C2
:10098000002101F02FFB22792346032A28BF0322EE
:1009900003F8042F28460222202101F023FB62796C
:1009A0002346072A28BF072203F8052F28460322DB
:1009B000222101F017FBA2792346072A28BF07222C
:1009C00003F8062F28460322252101F00BFB2846B9
:1009D00004F108031022282101F004FB382038BD5F
:1009E0002DE9F04FFFB01FAE0CAD40F279128046FA
:1009F0000F463046002100F017FD4822002128460E
:100A000000F012FD00F060FD574B4FF47A72B0FB1E
:100A1000F2F0186093E80700012385E807002B74C3
:100A20000DF1520000236B74FFF70AFF032385F8D2
:100A30002030E92385F8213006AB18464B4903F0F6
:100A400029FA162228643146284685F83C20FFF70B
:100A500091FF10AB044601460822304601F0C2FA6D
:100A60000822A1180DF14103304601F0BBFA0DF147
:100A70004203082204F11001304601F0B3FA11AB31
:100A8000202204F11801304601F0ACFA12AB4022EA
:100A900004F13801304601F0A5FA14AB082204F144
:100AA0007801304601F09EFA0DF15103082204F15D
:100AB0008001304601F096FA04F1880A0DF15209DE
:100AC00004F5847B4B465146082230460AF1080A59
:100AD00001F088FAD34509F10109F3D119AB0822D5
:100AE0005946304601F07EFA04F588744FF000094B
:100AF00095F834304B4510D84FF0000995F83C304C
:100B00004B4515D92B6C21464B440822304601F049
:100B100069FA083409F10109F0E7AB6B21464B444F
:100B20000822304601F05EFA083409F10109DFE7D6
:100B3000E31DC3F3CF03F97E0593002304960393CB
:100B4000BB7E0293193701230093019704A3D3E9D5
:100B50000023404601F016F87FB0BDE8F08F00BFDB
:100B60009E6AC421818A46EE882500204C400008F8
:100B7000014B1870704700BF94250020F0B52E4B34
:100B80001C7B85B02CB12D4B0E221A81002005B0A4
:100B9000F0BD2B4A1068516802AB03C308230DEB6C
:100BA00003022849284803F057F9054630B9234B7A
:100BB00026480A221A8100F03FFCE7E70369B3F5F3
:100BC000E02F07D91D4A22480B211181194600F058
:100BD00033FCDBE7418B40F2E932914206D0174B00
:100BE0000C2018811B4800F027FCCFE71A4A164951
:100BF0000244103B20469E1A00F06AFC324607462B
:100C000005F11801204600F063FCAB689F4202D159
:100C1000EB6898420AD0094B0D221A8100903B469E
:100C2000EA68A9680D4800F007FCAFE70C4800F03F
:100C300003FC0120ABE700BFC83500208825002059
:100C40003C3F0008DCFF060000000108443F0008AC
:100C5000503F0008623F00080800FFF7803F00088F
:100C6000A93F00082DE9F04FAFB006AF80460D4612
:100C700000F02EFF044600286CD12B7E022B18D1E9
:100C8000EB8A012B15D100F01FFC8146FFF7C0FD58
:100C90004FF4C873BF4EB0FBF3F209F5167902FBAF
:100CA0001300EB7E19FA80F0306093B9BA4B002242
:100CB0001A70A437BD46BDE8F08F07F10C031C4441
:100CC0000094002308224FEAC901284600F0EEFFF5
:100CD0004C46AB8A013BA3425FFA84F90BD904F17D
:100CE0000109B9F1110FE8D1AC4BAD4A40F239110D
:100CF000AC4803F083F807F11C00FFF7A1FD224682
:100D000007F11C0107F10C0003F096F803460028D8
:100D1000CCD1B9F1100F07D09F4B83F80090336806
:100D2000A3F516733360C4E707F1A002014602F889
:100D3000950D28460092072200F0B8FFF97A7F2926
:100D400004DD994B964A4FF4A871D1E7404600F074
:100D5000A3FEAEE7EB8A052B00F02E8106D8012B0F
:100D6000A7D129464046FFF73BFEA2E7282B3DD0FE
:100D7000302B9ED16B7E8D4C0133627BDBB2934274
:100D8000EA4640F00081EA7E237B9A4240F0FB80F5
:100D900007F1A003002623F8846D1022009331464A
:100DA0000123284600F082FFB5F81480A8F102085C
:100DB0001FFA88F808F1030323F003030A3323F032
:100DC0000703ADEB030D0DF1180933469BB2B11CBF
:100DD00098454FEAC10106F101066DDD4B440093D1
:100DE00008220023284600F061FFEEE7AB8A013BB2
:100DF0009BB2C92B3FF65DAF6C4E347B4CBB06F10A
:100E00000C030093082223462146284600F04EFF9B
:100E1000AB8A04F10109013BE4B29C424FEAC901EB
:100E200009DA0E343444009400230822284600F0E6
:100E30003DFF4C46ECE700230022C6E900230023D7
:100E4000B36086F8D730C6F8D830337B0BB9EB7E69
:100E50003373002407F11C0607F10C030822214616
:100E60003046FC603C617C6101F0BCF83B7C04F1E5
:100E70000109A3424FEAC90107D97B69082223442B
:100E8000304601F0AFF84C46F0E7C1F3CF01002344
:100E9000E87E059104960393AB7E029319352823CF
:100EA00001460093019539A3D3E90023404600F0A1
:100EB00069FEFFF7D5FCFCE694F8D70000F076FA5F
:100EC000D4F8D83006461BB994F8D70000F07EFA63
:100ED000D4F8D83043449E4204D294F8D70001306D
:100EE00000F074FA324B4FEA980B0025AAB25A452B
:100EF000104616DA5AB994F8D72042B9D4E900124C
:100F00000A4304D1D9F800201A600135EEE72268BF
:100F100059F820107B6002EB800000F037FA7B6804
:100F2000F3E7D4E90023D4F8D85012EB080043F1DA
:100F30000001C4E90001454494F8D700C4F8D85032
:100F400000F034FA854209D394F8D730013384F89D
:100F5000D730D4F8D8309E1BC4F8D860B8F1FF0F52
:100F60000ADC134B00201968207300F00FFAFFF71A
:100F700005FE08B1FFF7FCFB23680E4A9B0A01330C
:100F800013810023A360D54693E600BF2641727209
:100F9000DF25D7B79C35002099350020B83F0008E1
:100FA000644000081140000833400008C8350020A4
:100FB0000025002088250020BFF34F8F0549064BF0
:100FC000CA6802F4E0621343CB60BFF34F8F00BFE7
:100FD000FDE700BF00ED00E00400FA0508B54FF0A2
:100FE00000530B4A196891420AD10A4A597D11707F
:100FF00009481B7D0373C92208490E3000F002FA2C
:10100000E02200214FF00050BDE8084000F00CBA8B
:101010009AAD44C594250020C83500201600002054
:1010200030B5204C2049214885B00223002563714A
:1010300001230622ADF80C508DF80B308DF80C30E2
:101040004FF005134B60ADF808208DF80A2001F031
:1010500083FD174B019500931649174B17484FF422
:10106000805200F0E3FC164B1978254611B1134865
:1010700000F012FD00F028FA0446FFF7C9FB4FF418
:10108000C87304F51674B0FBF3F202FB13000D4BAA
:1010900014FA80F0186002F029FB08B10F232B81AD
:1010A00005B030BD8825002004250020B83600207A
:1010B000ED08000898250020650C0008A0350020E8
:1010C000942500209C3500202DE9F04F96A7D7E904
:1010D00000670FF25C29D9E900898F4C93B0DFF8E3
:1010E00058B2DFF858A2204600F098FD0CAD0790EA
:1010F00098B310220021284600F096F9079B197B2F
:101100004FF0000261F3030219468DF8302051F8C8
:10111000040F49680EAA03C21B680D9A63F31C02F0
:101120009DF830300D9243F020038DF830300023CD
:101130002A461946584601F01FFD079030B920464F
:1011400000F070FD079B8AF80030CCE79AF8003079
:10115000072B40DC01338AF8003018220021284692
:1011600000F062F9DFF8D0B1DFF8D4A1002319460E
:101170002A46584601F028FD014680BB102208A8E7
:1011800000F052F9DAF8143083F48053CAF81430BE
:1011900000F09CF90B4612A9024611E903000DF17B
:1011A000240E8EE803009DF83410C1F30300890675
:1011B0004CBF0E99BDF838108DF82C0046BFC1F316
:1011C0001C0141F00041C1F30A010891204608A921
:1011D00000F06EFFCAE7204600F024FDBDE7204680
:1011E00000F076FC824600284AD1DFF858B100F0C2
:1011F0006BF9DBF80030984242D300F065F90790B4
:10120000FFF706FB079A8DF820A04FF4C87302F58C
:101210001672B0FBF3F101FB130012FA80F0CBF869
:101220000000DFF824B19BF8001011B901238DF8FC
:10123000203028460791FFF703FB0799C1F1100AF8
:101240005FFA8AFABAF1060F28BF4FF0060A524633
:1012500029440DF1210000F0D5F80AF101030493AF
:1012600008AB0393182302932C4B019301230093A3
:1012700032463B46204600F02DFC00238BF8003020
:1012800000F022F9264ADFF8C4A01368C31AB3F5A8
:101290007A7F32D3106000F019F902460B462046DF
:1012A00000F0C6FC204600F013FC30B39AF80C3076
:1012B000DFF89CB0002B14BF032302238BF805300A
:1012C00000F002F94FF47A732946B0FBF3F0CBF843
:1012D00000005846FFF74EFB182307300293114BCE
:1012E0000193C0F3CF0040F255130490009303958F
:1012F00042464B46204600F0EDFB9AF80C300BB10D
:10130000FFF7AEFA9AF80C30002B7FF4E8AE13B07A
:10131000BDE8F08FAFF30080A035002098350020A5
:10132000A8360020AC360020401DA12026812A0BC3
:10133000F1C6A7C1D068080FB8360020AD3600202E
:10134000000402409C35002099350020C83500205B
:101350008825002070B502F04DF8094C094E207028
:10136000002530682378834208D902F03DF83368BD
:1013700005440133B5F5803F3360F2D370BD00BF43
:10138000B4360020B036002002F0E4B807B502AB56
:1013900000F1006043F8041D0422194600F5803076
:1013A00002F06EF803B05DF804FB0000054B1A680C
:1013B000054B1B789B1A834202D9104402F014B8E3
:1013C00000207047B0360020B436002038B5074DF5
:1013D00004462868204402F00FF828B92868204401
:1013E000BDE8384002F020B838BD00BFB03600205C
:1013F000022802BF024B4FF080529A61704700BF33
:101400000004024010B50023934203D0CC5CC454C6
:101410000133F9E710BD000002460346981A13F99C
:10142000011B0029FAD1704702440346934202D0BF
:1014300003F8011BFAE770470FB4002004B07047AF
:101440000EB4002003B07047FEE7000000B59BB06B
:10145000EFF3098168226846FFF7D4FFEFF30583B5
:10146000034B9A6B9A6A9A6A9A6A9A6A9B6AFEE72F
:1014700000ED00E000B59BB0EFF3098168226846FB
:10148000FFF7C0FFEFF30583044B9A6B9A6A9A6AE1
:101490009A6A9A6A9A6A9B6AFEE700BF00ED00E0CA
:1014A00000B59BB0EFF3098168226846FFF7AAFFF9
:1014B000EFF30583034B5A6B9A6A9A6A9A6A9A6A9F
:1014C0009B6AFEE700ED00E002F07CB802F056B83F
:1014D00030B5084D0A4491420BD011F8013B092464
:1014E0005840013CF7D040F300032B4083EA500002
:1014F000F7E730BD2083B8ED0246006848B10368C5
:101500001360D388118901339BB29942D38038BFCD
:101510001381704770B588B00D4604462022002123
:101520006846FFF781FF20460495FFF7E5FF054673
:1015300058B16B46044608AE1A4603CAB242206050
:101540006160134604F10804F6D1284608B070BD66
:101550002DE9F04130B9274B274A40F2C5312748E1
:1015600002F04CFC0B7C23B9254B234A40F2C631D8
:10157000F5E7C66986B9C161BDE8F081002B29DABB
:10158000930CAB4229D1B44201D10C60F3E7C8F807
:1015900000100C60BDE8F0814B6823F06047BD0C83
:1015A0004FEAD37EC3F3807C15EA230538BF3D465E
:1015B000B04634466368BEEBD37F23F06042DDD192
:1015C000974203D1C3F380739C450AD1974205E04B
:1015D0001C46EFE7AA4206D013469D422CBF0023CB
:1015E0000123002BCFD12368A046002BF0D121602E
:1015F000BDE8F081384300082C410008F0430008A2
:101600001144000808B5034A034B044840F25E3118
:1016100002F0F4FB08410008B0430008F043000862
:1016200008B503680B60C388016033B9044B054AF1
:1016300005484FF4C76102F0E1FB013BC38008BDE0
:10164000804300087C410008F043000870B50C4658
:1016500000F10C05616831B9E38A61F30903E382A3
:101660000020002170BD0E682846FFF7D9FF666094
:10167000F0E7000008B5426832B10B4B0B4A0C484A
:1016800040F22F4102F0BAFBC37DC3F38401013164
:1016900061F38603C375C38A62F30903C3821B0A1D
:1016A00062F3C713C37508BDCC4300083841000876
:1016B000F04300082DE9F047089E32B91F4B204A3D
:1016C000204840F2395102F099FB01F007054FEA3A
:1016D000D6082A4406F0070600EBD1004FF47F49F4
:1016E000954201D1BDE8F08705F0070E06F0070A24
:1016F000D645774638BF5746C7F10807511BEC0857
:101700008F4228BF0F46045D08EBD60104FA0EF4A1
:1017100013F801C029FA07FE24FA0AF45FFA8EFED4
:101720008CEA04044EFA0AFE04EA0E048CEA040C65
:1017300003F801C03D443E44D2E700BF4C430008DB
:1017400050410008F04300082DE9F04106460F46DD
:1017500000254FF6FF7441F221082A4630463946EB
:10176000FEF73EFDC0B284EA0024082314F4004FC3
:101770004FEA4404A4B203F1FF3318BF84EA08041B
:1017800013F0FF03F2D10835402DE6D12046BDE825
:10179000F081000010B50A4441F22104914200D1C9
:1017A00010BD11F8013B80EA0320082310F4004F1C
:1017B0004FEA400080B203F1FF3318BF604013F0DE
:1017C000FF03F3D1EAE700002DE9F04F85B08A4628
:1017D0008DE80C00BDF83C40814630B9494B4A4A7F
:1017E00040F26E31494802F009FB11F0604F04D01D
:1017F000474B454A40F26F31F4E7009B002B7ED007
:1018000024B10E9B002B7AD0072C28D809F10C00AC
:10181000FFF772FE054628B96FF00205284605B0AD
:10182000BDE8F08F14220021FFF7FEFD22460E993D
:1018300005F10800FFF7E6FD631C2B74009B1B7885
:101840002C4403F01F0363F03F0323724AF000436C
:101850006B6029464846FFF77BFE0125DEE7019BCA
:101860001B0A4FF00008029300F10C034FF0800BAD
:101870004646454603930398FFF73EFE0746002879
:10188000CAD014220021FFF7CFFDB6BB9DF804306B
:101890003B729DF808307B7202220E9B711E194428
:1018A000B4420AD9B8180132D2B211F801EF80F867
:1018B00008E00136072AB6B2F2D1009B197801F090
:1018C0001F01B44208BF4FF0400BB81841EA48115D
:1018D0004BEA0103037201324AF000437B603A7421
:1018E00039464846FFF734FE0135B4422DB288F040
:1018F00001084FF0000BBED190E70022CDE76FF05A
:1019000001058BE7384300081C410008F04300083C
:101910005C4300082DE9F0471E46CB8A9146C3F38D
:101920000902062A80460F4619D013460021B0B29C
:101930008DB25A1992B2052A09D9A84210D8FA8A4A
:10194000034463F30902FA820120BDE8F087A8424C
:10195000F3D93A4419F8014094760131E8E70025BB
:10196000FB8A7C68C3F30900821F1C23B2FBF3FAD5
:1019700003FB1A2A1FFA8AF27CB301212368002B89
:1019800039D1B31F03441C20B3FBF0F301339BB2E6
:1019900099420CD2BAF1000F09D14046FFF7ACFDD5
:1019A00008B1C0F800A0206008B304460022B6B217
:1019B0004FF0000AB54230D2691E49441346E01880
:1019C00001339BB211F801EF80F804E001351C2BC4
:1019D000ADB214D0AE42F2D8ECE74046FFF78CFD32
:1019E000044608B1002303607C60002CDED16FF058
:1019F0000200BDE8F087013189B21C46BEE7AE4265
:101A0000D8D94046FFF778FD08B1C0F800A02060A3
:101A10000028ECD004460022CCE7FB8AC3F309027D
:101A2000164466F30903FB828EE70000F8B50E4604
:101A300015461F46044628B9144B154A15484F2130
:101A400002F0DCF924220021FFF7EEFC069B636024
:101A5000079B23626A094FF6FF739A424FF000001A
:101A600028BF1A46A7602070A061E06197B204F118
:101A70000C05824205D100232B6027826382A3825A
:101A8000F8BD2E60013035462036F2E734430008B9
:101A9000A8400008F043000808B528B9084B094AD7
:101AA0007321094802F0AAF9037823B94BB2002B3D
:101AB00001DD017008BD054B024A7D21F1E700BF41
:101AC00038430008B4400008F04300087C42000896
:101AD000007870472DE9F7430D9EBDF828900B9DC7
:101AE0009DF83040BDF8388007461946104616B9B3
:101AF000B8F1000F43D11F2C41D83B78D3B9B8F1CE
:101B0000070F39D839F0030339D1424631464FF631
:101B1000FF70FFF73FFE4FEA092920F0010009F4AA
:101B20004079400449EA0464400C44EA40244FF6FA
:101B3000FF730DE043EA0923B8F1070F43EA046499
:101B4000F5D9FFF701FE42463146FFF723FE034673
:101B50008DE840012A4621463846FFF735FE0DB98B
:101B6000FFF750FD2B780133DBB21F2B88BF00231A
:101B70002B7003B0BDE8F0836FF00300F9E76FF05E
:101B80000100F6E72DE9F7430E9F0B9D9DF8348089
:101B9000BDF83C6081469DF8300007B9C6BB1F28E0
:101BA00036D899F800E0BEF1000F34D00C0244F0B2
:101BB00080049DF8281044EAC83444EA014444EA09
:101BC0000E04072E44EA006415D919461046FFF7A3
:101BD000BBFD32463946FFF7DDFD0346019600970F
:101BE0002A4621464846FFF7EFFDB8F1010F0CD118
:101BF00025B9FFF707FD4FF6FF73EFE72B780133A9
:101C0000DBB21F2B88BF00232B7003B0BDE8F0832D
:101C10006FF00100F9E76FF00300F6E7C06900B16B
:101C200004307047C1690B68C3610C30FFF7F8BC22
:101C30002DE9F84FD0F818A0DFF86C80054616465D
:101C40001F4654464FF0000900F10C0B0CB9BDE8DB
:101C5000F88FD4E90223B21A67EB0303994508BF52
:101C600090451FD2AB699C42214628460DD1FFF713
:101C7000EDFCAB691B68AB6121465846FFF7D0FC11
:101C8000AC692346A2461C46E0E7FFF7DFFC236869
:101C9000CAF8003021465846FFF7C2FC5446DAF82D
:101CA0000030EFE72368EDE780841E002DE9F04F58
:101CB0008BB00D4614460793DDF8509082460028FD
:101CC00000F06481B9F1000F00F06081531E3F2BDA
:101CD00000F25C81012A03D1079B002B40F0568162
:101CE000BAF81460F6000023B5420893099380F017
:101CF00053812B199E420AD2761B16F0FF0607D19C
:101D0000AB4BAC4A40F26751AB4802F077F826463D
:101D1000DAF80C3023B9DAF81030002B00F0A58087
:101D20002F2D31D8C5F1300846454FF000032CBFA8
:101D30005FFA88F8B0460093294608AB4246DAF8C5
:101D40000800FFF7B7FCA6EB08074544FFB2BAF856
:101D5000143003F10053063BDB000293DAF80C3039
:101D600005934FF0300B059B002B51D087B9DAF863
:101D70001000002861D0002F5FD0AB4550D98F4BA9
:101D80008C4A40F2A651BFE737464FF00008DEE725
:101D9000029B23B98A4B874A4FF4B161B4E7029B97
:101DA000E02B28BFE02306935B44AB4204931DD98C
:101DB0005B1B9F4226BFDBB203930397AB4504D95D
:101DC0007E4B7C4A40F291519EE70598CDF8008009
:101DD00008ABA5EB0B01039A0430FFF76BFC039BE8
:101DE0009844FF1A1D445FFA88F8FFB2049B9B4594
:101DF00004D3744B6F4A40F29B5185E7029B069ACD
:101E0000DDF810B09B1A0293059B1B680593AAE7A7
:101E1000029BBB42ABD26C4B664A40F2A15173E7C6
:101E2000CDF800803A46A5EB0B0108ABFFF742FC6A
:101E3000B8443D445FFA88F80027BAF81430B5EB8F
:101E4000C30F04D9614B5B4A40F2B1515CE7B8F172
:101E5000400F04D95E4B574A40F2B25154E767B184
:101E60005C4B544A40F2B3514EE70093324608AB04
:101E70002946DAF80800FFF71DFC731E3F2B35B228
:101E800001D8A64204DD544B544A40F235213BE7C9
:101E900060070AD00AAB03EBD401624211F8083C98
:101EA00002F00702134101F8083C082C21D9102C3C
:101EB00021D9202C8CBF08230423079A002A6DD037
:101EC000B4EBC30F6CD0082C04F1FF3215D89DF889
:101ED000203023FA02F2D10706D54FF0FF3202FA82
:101EE00004F423438DF820309DF8203089F8003029
:101EF0004EE00123E1E70223DFE7102C11D8BDF803
:101F0000203023FA02F2D20706D54FF0FF3202FA50
:101F100004F42343ADF82030BDF82030A9F8003098
:101F200036E0202C0ED8089921FA02F2D30705D505
:101F30004FF0FF3303FA04F40C430894089BC9F8EC
:101F4000003025E0402C1CD0DDE9086730463946DA
:101F5000FEF746F9002100F0010050EA01030BD022
:101F6000224601200021FEF747F9404261EB410182
:101F700006430F43CDE90867DDE90823C9E90023DB
:101F800006E0174B154A4FF42071BDE66FF00105CE
:101F900028460BB0BDE8F08F1D46F9E7012CA3D011
:101FA000082CA1D9102CB7D9202CE5D8C6E700BF42
:101FB0008841000860410008F0430008AA41000879
:101FC00097410008CF410008F74100081E42000871
:101FD0004C420008644200087E420008E0400008CD
:101FE0007C42000830B585B030B9244B244A40F219
:101FF000B121244801F002FF23B9234B204A40F2CB
:10200000B221F6E7402A04D9204B1D4A40F2B621FE
:10201000EFE722B91D4B1A4A4FF42F71E9E700246C
:10202000012A0294039417D11B788DF808305307C6
:102030000AD004AB03EBD203554213F8084C05F069
:102040000705AC4003F8084C00910346002102A8A4
:10205000FFF730FB05B030BD082AE5D9102A03D8B8
:102060001B88ADF80830E2E7202A02D81B680293EB
:10207000DDE7D3E90045CDE90245D8E7B8420008DD
:10208000F4400008F0430008D34200087C420008F6
:1020900070B50C4600F10C05E16819B9A160216129
:1020A000A18270BD0E682846FFF7BAFAE660F3E732
:1020B0002DE9F04FD1F8009091B0C9F3C016044655
:1020C0000D46CDE90223002E50D0C9F3C03BC9F321
:1020D0000626B9F1000F80F29F8119F0C04F40F041
:1020E0009B812B7B002B00F09781BBF1020F03D06B
:1020F0002278B24240F0938109F07F02BBF1020FD7
:10210000059236D119F07F0FC9F30F2A01D10AF0D9
:10211000030A2B447606059A93F8038046EA0B4699
:1021200046EA82465FEAD81346EA0A06069300F0BA
:102130009A800022002310A961E90823059B0093DF
:1021400067685B4652462046B847002800F0888002
:10215000A7698FB9314604F10C00FFF7DBF9074698
:10216000D0B96FF0020011B0BDE8F08F4FF0020B54
:10217000AFE7C9F3074ACCE73B699E420DD03F6801
:10218000002FF9D1314604F10C00FFF7C3F90746DF
:102190000028E6D0A3693B60A761DDE90801FFF7ED
:1021A000D3FAB882F97D08F01F06C1F38401711AD1
:1021B00089B20FFA81FED7E90223BEF1000FB8BF42
:1021C00001F1200EC9F30461B8BF0FFA8EFE07912A
:1021D00052EA030100F02F81DDE90201801A61EB70
:1021E000030102460B469F480021994208BF9042D6
:1021F000C0F02181069B002B3FD0BEF1010F00F300
:102200001A8118F0400F38D0DDE90223C7E9022314
:10221000202200210DEB0200FFF706F9DDE9022381
:10222000CDE908232B1D0A932B7BADF836A0013B8B
:10223000DBB2ADF834309DF81C308DF83A309DF8A3
:1022400014308DF83B3020468DF838B08DF8396069
:10225000A36808A998473846FFF70CFA002082E7E0
:102260006FF00B007FE7A76917B96FF00C007AE7F2
:102270003B699E4296D03F68F6E7FB7DC8F340126B
:10228000B2EBD31F40F0CE80C3F38403B34240F0DF
:10229000CC8006992B7B4FEA981279B3D2073CD4B5
:1022A000032B40F2C580DDE90223C7E902232B7B23
:1022B000AE1D033BDBB23246394604F10C00FFF79A
:1022C00029FB002808DA39462046FFF7BFF93846CF
:1022D000FFF7D0F9032046E7AB883B832A7B033A1C
:1022E000D2B2B88A3146FFF755FAFB7DB882DA439D
:1022F000C2F3C01262F3C713FB75AFE76AB92E1DB4
:10230000013BDBB23246394604F10C00FFF702FB19
:102310000028D8DB2A7B013AE2E7FA8AC2F30902F5
:10232000013B052AD9B250D8281D002399420AD969
:1023300007EB020E013210F801CB8EF81AC0013300
:10234000062ADBB2F2D1DDE902898B4207F11A02DB
:10235000CDE908890A9238BF04337A680B9234BFFA
:102360005B1900230C93FB8AADF836A0C3F3090375
:1023700019449DF81C308DF83A309DF814308DF8D2
:102380003B300023ADF834108DF838B08DF839604B
:102390007B602A7BB88A013A291DFFF7FBF93B8B4A
:1023A000B882834203D1A36808A92046984708A9A8
:1023B0002046FFF76DFE3846FFF75CF9B88A3B8B85
:1023C000984214BF11200020CDE6786810B34FF07A
:1023D000060E03689BB9A2EB0E021B2A13D8033228
:1023E000024405F1040E1F309942ACD91EF801CB0E
:1023F00002F801CF01339042DBB2F5D1A3E70EF131
:102400001C0E1846E5E7184B184A194840F2B3115C
:1024100001F0F4FC034696E76FF00900A3E66FF0C5
:102420000A00A0E66FF00D009DE66FF00E009AE640
:102430006FF00F0097E6FB7D68F386036FF3C71319
:10244000FB7539462046FFF701F9069B002B7FF408
:10245000D8AEFB7DC3F38402013262F38603FB75C1
:1024600003E700BF80841E00E8420008CC4000085B
:10247000F04300082DE9F041504EB04240F0898011
:102480004F4CDFF840E1256C45F000752564256E62
:1024900045F000752566246E846AD4F8007207EA58
:1024A0000E0747F00107C4F80072D4F8005205EA9D
:1024B0000E0545F0010545EA0121C4F80012002A85
:1024C00069D00021C4F81C120F46C4F80412C4F8E5
:1024D0000C12C4F8141204EBC10501311C29C5F813
:1024E0004072C5F84472F6D14FF0000E4FF0010C67
:1024F000964514D1826AD2F80032B04223F001032B
:10250000C2F8003257D12E4B1A6C22F000721A64B6
:102510001A6E22F000721A661B6EBDE8F0819F7879
:102520001D8817F0010F18BFD4F804820CFA05F1CA
:102530001CBF41EA0808C4F8048217F0020F1EBF4E
:10254000D4F80C8241EA0808C4F80C827F0742BF25
:10255000D4F814720F43C4F8147204EBC5055F6815
:10256000C5F840729F68C5F84472D4F81C522943DC
:10257000C4F81C120C330EF1010EB9E7846A002175
:10258000C4F81C12C4F80412C4F80C12C4F81412D3
:10259000AAE7002AF2D1836A0022C3F84022C3F8D6
:1025A0004422C3F80422C3F814220122C3F80C22E7
:1025B000C3F81C229EE7BDE8F08100BFB8360020BA
:1025C000003802400000FFFF184A916A08B58B6886
:1025D0008B6013F0010105D013F00C0F14BF4FF402
:1025E00080310121D80506D513F4406F14BF41F4A2
:1025F000003141F00201D80306D513F4402F14BF77
:1026000041F4802141F00401D3690BB10748984798
:10261000202383F311880021054800F0E9FD002301
:1026200083F31188BDE8084001F076B8B836002081
:10263000C036002038B5124CA36ADD68AA0712D054
:102640005A6922F002025A61A36913B1012120469E
:102650009847202383F3118800210A4800F0C8FD21
:10266000002383F31188EB0606D5A36A1021D960F5
:10267000236A0BB102489847BDE8384001F04CB8D6
:10268000B8360020C836002038B5124CA36A1D6940
:10269000AA0712D05A6922F010025A61A36913B135
:1026A000022120469847202383F3118800210A48FD
:1026B00000F09EFD002383F31188EB0606D5A36A84
:1026C00010211961236A0BB102489847BDE83840D0
:1026D00001F022B8B8360020C836002038B50F4CBB
:1026E000A36A5D685D602A070AD5032222701A6812
:1026F00022F002021A60636A13B100212046984753
:102700006B0706D5A36A9969236A13B109040348C4
:102710009847BDE8384000F0FFBF00BFB836002042
:1027200010B50F4C204600F005FA0E4BA3620B21AA
:10273000132000F0E7F90B21142000F0E3F90B213E
:10274000152000F0DFF90B21162000F0DBF9002343
:1027500020461A460E21BDE81040FFF78BBE00BF91
:10276000B836002000640040114B984210B5044672
:1027700009D1104B1A6C42F000721A641A6E42F0C2
:1027800000721A661B6EA36A01221A60A36A5A6855
:10279000D20707D5626851681268D9611A60064A83
:1027A0005A6110BD0121082000F056FCEEE700BF81
:1027B000B8360020003802405B87010003291AD890
:1027C000DFE801F0020A0F14836A9B6813F0E05FF0
:1027D00014BF012000207047836A9868C0F38060AE
:1027E0007047836A9868C0F3C0607047836A9868CE
:1027F000C0F30070704700207047000010B5032937
:102800001FD8DFE801F0021F2327816A8B68C3F31A
:102810000163183301EB0313107881061ED5546849
:10282000C0F30011490041EAC40141F0040100F085
:102830000F00586090689860D268DA6041F001013A
:10284000196010BD836A03F5C073E5E7836A03F579
:10285000C873E1E7836A03F5D073DDE79488C0F3BA
:102860000011490041EA4451E1E7000001290CD080
:1028700003D3022910D000207047836ADA689207D8
:1028800001D1186903E001207047836AD86810F00D
:10289000030018BF01207047836AF2E710B539B909
:1028A000836AD96889071BD11B699B0704D110BDB6
:1028B000012915D0022948D1816AD1F8C031D1F857
:1028C000C401D1F8C8411461D1F8CC41546120242D
:1028D0000C610C69A40717D14C6944F0100412E094
:1028E000816AD1F8B031D1F8B401D1F8B84114619E
:1028F000D1F8BC4154612024CC60CC68A40703D13A
:102900004C6944F002044C6111795C0864F30411D1
:102910009C0864F34511117189064BBF91681189B8
:10292000DB085B0D4CBF63F31C0163F30A011379F1
:1029300048BF916060F3030313714FEA10234FEA1D
:10294000104058BF11811370508010BD00230449FE
:102950001A465A50C8180833802B4260F9D1704784
:10296000E4360020026843681143016003B1184750
:1029700070470000024AD36843F0C003D360704739
:1029800000100140024AD36843F0C003D36070478F
:10299000004400402DE9F041D0F85C64F7683368EA
:1029A000DA0505469CB20DD5202383F311884FF438
:1029B00000710430FFF7D6FF6FF48073336000239B
:1029C00083F31188202383F3118805F1040814F0A0
:1029D0002F0333D183F31188380615D5210613D57B
:1029E000202383F3118805F1380000F027FA00282E
:1029F00046DA0821281DFFF7B5FF4FF67F733B40ED
:102A0000F360002383F311887A060ED563060CD594
:102A1000202383F31188EA6C2B6D9A4202D12B6C30
:102A2000002B2FD1002383F31188D5F86424D368B9
:102A3000002B31D01069BDE8F0411847230713D0AF
:102A400014F0080F0CBF00218021E00748BF41F0BF
:102A50002001A20748BF41F04001630748BF41F48D
:102A600080714046FFF77EFFA406736805D595F890
:102A700060142846194000F083FA3468A4B2A6E72F
:102A80007060BEE727F040073F041021281D3F0C6F
:102A9000FFF768FFF760C5E7BDE8F08108B50348B8
:102AA000FFF778FFBDE8084000F036BE643700202D
:102AB00008B50348FFF76EFFBDE8084000F02CBEE4
:102AC000CC3B002010B5094C094A2046002100F0FB
:102AD00035FA084BC4F85C34074C084A00212046FC
:102AE00000F02CFA064BC4F85C3410BD64370020AB
:102AF0007529000800100140CC3B00208529000802
:102B00000044004000F1604300F01F02400903F55B
:102B1000614309018000C9B200F1604083F80013ED
:102B200000F5614001239340C0F880310360704795
:102B3000FFF7F6BD00F10802012303708260002355
:102B4000C26000F110024360026142618361C361AF
:102B5000036243627047000010B52023044683F3EC
:102B60001188022303704160FFF7FEFD03232370E9
:102B7000002383F3118810BD2DE9F0411F46044660
:102B80000D461646202383F3118800F108082378A8
:102B9000042B0ED029462046FFF710FE48B12046F0
:102BA00032462946FFF72AFE002080F31188BDE84F
:102BB000F0813946404600F0FFFA0028E7D00023B4
:102BC00083F31188BDE8F0812DE9F0411F460446EA
:102BD0000D461646202383F3118800F11008237850
:102BE000042B0ED029462046FFF740FE48B1204670
:102BF00032462946FFF752FE002080F31188BDE8D7
:102C0000F0813946404600F0D7FA0028E7D000238B
:102C100083F31188BDE8F081F8B51546826806692E
:102C2000AA420B46816938BF8568761AB5420446C8
:102C300007D218462A46FEF7E5FBA3692B44A36199
:102C40000DE011D932461846FEF7DCFBAF1B3A46C1
:102C5000E1683044FEF7D6FBE2683A44A261A3681B
:102C60005B1BA3602846F8BD18462A46FEF7CAFB40
:102C7000E368E4E783682DE9F04104469342154692
:102C8000266938BF85684069361AB5420F4606D2B4
:102C90002A46FEF7B7FB63692B4463610DE012D946
:102CA0003246A5EB0608FEF7ADFB4246B919E068CF
:102CB000FEF7A8FBE26842446261A3685B1BA36065
:102CC0002846BDE8F0812A46FEF79CFBE368E4E76E
:102CD00010B50A440024C361029B00604060846018
:102CE000C160816141610261036210BD08B5826902
:102CF0004369934201D1826882B98268013282605D
:102D00005A1C42611970426903699A4201D3C3682F
:102D10004361002100F060FA002008BD4FF0FF3051
:102D200008BD000070B5202304460E4683F31188C9
:102D3000A568A5B1A368A269013BA360531CA36168
:102D400015782269934224BFE368A361E3690BB15C
:102D500020469847002383F31188284670BD3146EA
:102D6000204600F029FA0028E2DA85F3118870BDC8
:102D70002DE9F74F05460F4690469A46D0F81C902D
:102D8000202686F311884FF0000B144664B12246CA
:102D900039462846FFF740FF034668B951462846A2
:102DA00000F00AFA0028F1D0002383F31188A8EB81
:102DB000040003B0BDE8F08FB9F1000F03D001901B
:102DC0002846C847019B8BF31188E41A1F4486F3F9
:102DD0001188DBE7C16081614161C3611144009BDF
:102DE000006040608260016103627047F8B504468C
:102DF0000E461746202383F31188A568A5B1A36862
:102E0000013BA36063695A1C62611E702369626999
:102E10009A4224BFE3686361E3690BB12046984797
:102E2000002080F31188F8BD3946204600F0C4F92F
:102E30000028E2DA85F31188F8BD00008369426951
:102E40009A4210B501D182687AB9826801328260F3
:102E50005A1C82611C7803699A4201D3C36883615A
:102E6000002100F0B9F9204610BD4FF0FF3010BD31
:102E70002DE9F74F05460F4690469A46D0F81C902C
:102E8000202686F311884FF0000B144664B12246C9
:102E900039462846FFF7EEFE034668B951462846F4
:102EA00000F08AF90028F1D0002383F31188A8EB01
:102EB000040003B0BDE8F08FB9F1000F03D001901A
:102EC0002846C847019B8BF31188E41A1F4486F3F8
:102ED0001188DBE7026843681143016003B11847BA
:102EE000704700001430FFF743BF00004FF0FF337E
:102EF0001430FFF73DBF00003830FFF7B9BF0000C6
:102F00004FF0FF333830FFF7B3BF00001430FFF746
:102F100009BF00004FF0FF311430FFF703BF00007E
:102F20003830FFF763BF00004FF0FF323830FFF753
:102F30005DBF000000207047FFF7C4BD37B50F4BE1
:102F40000360002343608360C3600123044603746D
:102F5000154600900B464FF4007200F15C011430EE
:102F6000FFF7B6FE00942B464FF4007204F517717C
:102F700004F13800FFF72EFF03B030BD2C440008E9
:102F800038B5C36904460D461BB904210844FFF750
:102F9000A1FF294604F11400FFF7A8FE002806DA75
:102FA000201D4FF48061BDE83840FFF793BF38BD66
:102FB000024B00221B605B609A6070473440002027
:102FC000002303748268054B1B6899689142FBD209
:102FD0005A680360426010605860704734400020B7
:102FE00008B5202383F31188037C032B05D0042B21
:102FF0000DD02BB983F3118808BD436900221A60F4
:103000004FF0FF334361FFF7DBFF0023F2E790E867
:103010000C001A6002685360F2E70000002303749A
:103020008268054B1B6899689142FBD85A68036017
:10303000426010605860704734400020054B1969A9
:103040000874186802681A605360186101230374D9
:10305000FDF7FABA3440002030B54B1C87B0054666
:103060000A4C10D023690A4A01A800F0DDF828466E
:10307000FFF7E4FF049B13B101A800F011F92369E5
:10308000586907B030BDFFF7D9FFF8E7344000209A
:10309000E12F000838B50C4D41612B6981689A68B1
:1030A0009142044603D8BDE83840FFF789BF18466F
:1030B000FFF786FF01232C61014623742046BDE8FB
:1030C0003840FDF7C1BA00BF34400020044B1A68F5
:1030D0001B6990689B68984294BF0020012070474C
:1030E0003440002010B5084C236820691A6822601B
:1030F0005460012223611A74FFF790FF0146206992
:10310000BDE81040FDF7A0BA3440002008B5FFF735
:10311000DDFF18B1BDE80840FFF7E4BF08BD0000BF
:103120008260022202740022427470478368A3F115
:103130007C0243F80C2C026943F83C2C426943F8AA
:10314000382C074A43F81C2CC26843F8102C022282
:1031500003F8082C002203F8072CA3F1180070478D
:103160006106000810B5202383F31188FFF7DEFF06
:1031700000210446FFF78EFF002383F311882046C9
:1031800010BD0000024B1B6958610F20FFF756BFAE
:1031900034400020202383F31188FFF7F3BF0000A1
:1031A00008B50146202383F311880820FFF754FF58
:1031B000002383F3118808BD49B1064B42681B699F
:1031C00018605A60136043600420FFF745BF4FF05A
:1031D000FF307047344000200368984206D01A68D8
:1031E0000260506059611846FFF7EABE7047000060
:1031F00038B504460D462068844200D138BD0368C6
:1032000023605C604561FFF7DBFEF4E7054B03F1EB
:1032100014025A619A614FF0FF32DA6100221A6299
:10322000704700BF34400020F8B503614FF0804381
:10323000C2605C6A194B1A46022952F8145F38BF03
:103240000221954206461F460AD1586198611C62C8
:103250000560456081600819BDE8F84000F0AABA31
:10326000186AAB68241A0C1902D3E41A2D6804E01A
:103270009C4202D2204400F0ABFAAB689C42F4D8E6
:103280006B68736035601E606E60B460A9684FF053
:10329000FF33091BA960FB61F8BD00BF344000206B
:1032A00010B41B4C234653F8141F814210D04168C0
:1032B00002680A60026851609A424FF00001C160E2
:1032C00003D0936881680B4493605DF8044B7047AA
:1032D0000A68626100209A425360C86003D15DF8B9
:1032E000044B00F06FBA93688868034493604FF012
:1032F0008042206A526A121A9342E6D9991A012929
:1033000098BF931C18445DF8044B00F061BA00BFED
:103310003440002000207047FEE7000070470000A6
:103320004FF0FF3070470000BFF34F8F024AD36861
:10333000DB03FCD4704700BF003C024008B5094BDA
:103340001B7873B9FFF7F0FF074B1A69002ABFBF5C
:10335000064A5A6002F188325A601A6822F4806282
:103360001A6008BD74400020003C024023016745FC
:1033700008B50B4B1B7893B9FFF7D6FF094B1A69B9
:1033800042F000421A611A6842F480521A601A68C8
:1033900022F480521A601A6842F480621A6008BDF2
:1033A00074400020003C0240072870B513D80B4A37
:1033B0000B4C137863B90B4E4FF0006144F82310A7
:1033C00056F823500133082B2944F7D101231370F9
:1033D00054F8200070BD002070BD00BF9840002050
:1033E0007840002054440008014B53F820007047F7
:1033F0005444000808207047072810B5044601D936
:10340000002010BDFFF7D0FF064B53F824301844BE
:10341000C21A0BB9012010BD12680132F0D1043B71
:10342000F6E700BF54440008072810B5044621D829
:10343000FFF77AFFFFF782FF0F4AF323D360C30041
:10344000DBB243F4007343F002031361136943F4E6
:1034500080331361FFF768FFFFF7A6FF074B53F8B0
:10346000241000F00DF9FFF783FF2046BDE810405F
:10347000FFF7C2BF002010BD003C024054440008CA
:103480002DE9F84312F00103154640D184182E4A65
:1034900094423CD82D4B1B6813F0010337D02C4CC1
:1034A000FFF74CFFF323E360FFF73EFF40F20127F5
:1034B000032D01D9830713D0254C0F46401A40F243
:1034C0000118EB1B0B44012B00EB0706236924D8E2
:1034D00023F001032361FFF74BFF0120BDE8F883D0
:1034E000236923F44073236123693B43236151F82B
:1034F000046B0660BFF34F8FFFF716FF03689E4211
:1035000008D0236923F001032361FFF731FF002076
:10351000BDE8F883043D0430CAE723F44073236117
:10352000236943EA08032361B94637F8023B338035
:10353000BFF34F8FFFF7F8FE3688B9F80030B6B208
:10354000B342BED0DDE700BFFFFF070800380240EE
:10355000003C0240084908B50B7828B153B9FFF781
:10356000EDFE01230B7008BD23B1BDE808400870D3
:10357000FFF7FEBE08BD00BF7440002070B500F02C
:10358000AFF90E4E4FF08043596A3368994210D21A
:103590000B4CD4E90023003243F10103C4E90023BA
:1035A000541843F10005316000F0A4F92046294683
:1035B00070BD034BD3E90023F2E700BF9C4000201D
:1035C000A040002008B5FFF7D9FF4FF47A7200231E
:1035D000FCF71EFE08BD00BF10B50244064B0439BF
:1035E000D2B2904200D110BD441C00B253F820006A
:1035F00041F8040FE0B2F4E750280040104B30B51A
:103600001C6F240407D41C6F44F400741C671C6FE7
:1036100044F400441C670B4C236843F4807323601C
:103620000244094B0439D2B2904200D130BD441C4F
:1036300000B251F8045F43F82050E0B2F4E700BF55
:1036400000380240007000405028004007B50122B9
:1036500001A90020FFF7C0FF019803B05DF804FB4B
:1036600013B50446FFF7F2FFA04206D002A90122DB
:1036700041F8044D0020FFF7C1FF02B010BD00006B
:1036800070470000074B45F255521A6002225A60FB
:1036900040F6FF729A604CF6CC421A60024B01224F
:1036A0001A70704700300040A9400020034B1B787F
:1036B0001BB1034B4AF6AA221A607047A9400020AA
:1036C00000300040034B1B689B0042BF024B0122AD
:1036D0001A70704774380240A8400020024B4FF027
:1036E00080721A60704700BF74380240014B18782E
:1036F000704700BFA8400020064A536823F001032A
:103700005360EFF30983683383F30988002383F35D
:103710001188704730EF00E010B5202383F3118843
:10372000104B5B6813F4006318D0F1EE103AEFF31E
:1037300009844FF0807344F84C3C0B4BDB6844F831
:10374000083CA4F1680383F30988FFF7BFFC18B1B4
:10375000064B44F8503C10BD054BFAE783F3118843
:1037600010BD00BF00ED00E030EF00E07106000882
:103770007406000870470000FEE70000084A094B85
:1037800009498B4204D3094A0021934205D370476B
:1037900052F8040F43F8040BF3E743F8041BF4E773
:1037A00034460008AC420020AC420020AC4200206D
:1037B00000F034B94FF08043002258631A610222AE
:1037C000DA6070474FF080430022DA6070470000F3
:1037D0004FF0804358637047FEE7000010B5174C68
:1037E000FFF7E6FBFFF712FD802215492046FFF7A1
:1037F00097FC012344F8180C0374124B124AD96841
:1038000021F4E0610904090C0A431049DA60CA682E
:1038100042F08072CA600E490A6842F001020A60F2
:103820001022DA77202283F82220002383F31188E4
:1038300062B60848BDE81040FFF794BC5C40002029
:103840007444000800ED00E00003FA05F0ED00E02C
:10385000001000E07C4400082DE9F84F1F4C4FF0A9
:103860000008656904F11407C1464FF08043266AD9
:103870005B6AAA689E1B96421DD34FF0200AAA6875
:10388000236AD5F80CB0134423622B68BB425F60F7
:10389000A6EB02066361C5F80C8001D1FFF792FF29
:1038A00089F311882869D8478AF311886569AB685C
:1038B0009E42E4D2D9E76269BA420CD09168236291
:1038C0008E1B9660A86802282CBF1818981CBDE8AB
:1038D000F84FFFF77DBFBDE8F88F00BF34400020F0
:1038E000EFF3118020B9EFF30583202282F31188D2
:1038F0007047000010B558B9EFF30584C4F308040D
:1039000014B180F3118810BDFFF700FC84F3118817
:1039100010BD00004B6843608B688360CB68C36058
:103920000B6943614B6903628B6943620B680360F7
:103930007047000008B51F4B1F481A6942F0FF028C
:103940001A611A6922F0FF021A611A691A6B42F0B1
:10395000FF021A631A6D42F0FF021A65174A1B6DC7
:103960001146FFF7D7FF164802F11C01FFF7D2FFFF
:10397000144802F13801FFF7CDFF134802F154015A
:10398000FFF7C8FF114802F17001FFF7C3FF1048AD
:1039900002F18C01FFF7BEFF0E4802F1A801FFF70C
:1039A000B9FF0D4802F1C401FFF7B4FFBDE80840BC
:1039B00000F09CB800380240000002409C4400081F
:1039C0000004024000080240000C024000100240C7
:1039D0000014024000180240001C024008B500F02C
:1039E000FDF9FFF7FBFEBDE80840FFF76BBE0000E6
:1039F000704700004FF0804310B51A69920708D550
:103A000000241C61202383F31188FFF725FF84F332
:103A10001188BDE81040FFF77FBE0000104B1A6C04
:103A200042F001021A641A6E42F001021A660D4A4F
:103A30001B6E936843F0010393604FF080435F2255
:103A40009A624FF0FF32DA6200229A615A63DA60BA
:103A50005A6001225A6108211A601C20FFF752B8EF
:103A600000380240002004E01E4B1A6962F0FF0299
:103A70001A611A69D2B21A614FF0FF301A695A6995
:103A8000586100215A6959615A691A6A62F0805274
:103A90001A621A6A02F080521A621A6A5A6A5862E4
:103AA0005A6A59625A6A1A6C42F080521A641A6E43
:103AB00042F080521A661A6E0B4A106840F4807009
:103AC0001060186F00F44070B0F5007F1EBF4FF417
:103AD000803018671967536823F40073536000F04F
:103AE0005DB900BF0038024000700040334B344ADB
:103AF0001A64344A4FF4404111601A6842F00102DE
:103B00001A601A689207FCD59A6822F003029A603C
:103B10002A4B19469A6812F00C02FBD1186800F083
:103B2000F90018609A601A6842F480321A600B68D3
:103B30009B03FCD54B6F43F001034B671F4B5A6F40
:103B40009007FCD5204A5A601A6842F080721A60C9
:103B50001C4A53685904FCD5184B1A689201FCD5CD
:103B60001A4A9A600322C3F88C200022C3F89420DA
:103B7000174B1A68174B9A42174B1BD1174A1168FB
:103B8000174A914216D140F203121A600B4B9A6801
:103B900042F002029A609A6802F00C02082AFAD1F6
:103BA0005A6C42F480425A645A6E42F480425A6619
:103BB0005B6E704740F20372E7E700BF00380240D7
:103BC0000004001000700040106041080090883828
:103BD000002004E011640020003C024000ED00E001
:103BE00041C20F41084A08B5536911680B4003F000
:103BF0000103536123B1054A13680BB1506898471C
:103C0000BDE80840FFF788BD003C0140E4360020D5
:103C1000084A08B5536911680B4003F00203536169
:103C200023B1054A93680BB1D0689847BDE80840B6
:103C3000FFF772BD003C0140E4360020084A08B599
:103C4000536911680B4003F00403536123B1054A23
:103C500013690BB150699847BDE80840FFF75CBD98
:103C6000003C0140E4360020084A08B55369116859
:103C70000B4003F00803536123B1054A93690BB16C
:103C8000D0699847BDE80840FFF746BD003C0140B9
:103C9000E4360020084A08B5536911680B4003F068
:103CA0001003536123B1054A136A0BB1506A984758
:103CB000BDE80840FFF730BD003C0140E43600207D
:103CC000174B10B55C691A68144004F478725A6195
:103CD000A30604D5134A936A0BB1D06A98476006CD
:103CE00004D5104A136B0BB1506B9847210604D5CD
:103CF0000C4A936B0BB1D06B9847E20504D5094A87
:103D0000136C0BB1506C9847A30504D5054A936C0E
:103D10000BB1D06C9847BDE81040FFF7FDBC00BF69
:103D2000003C0140E43600201A4B10B55C691A686B
:103D3000144004F47C425A61620504D5164A136D9E
:103D40000BB1506D9847230504D5134A936D0BB101
:103D5000D06D9847E00404D50F4A136E0BB1506E36
:103D60009847A10404D50C4A936E0BB1D06E9847C6
:103D7000620404D5084A136F0BB1506F98472304AF
:103D800004D5054A936F0BB1D06F9847BDE810403A
:103D9000FFF7C2BC003C0140E4360020062108B514
:103DA0000846FEF7AFFE06210720FEF7ABFE062110
:103DB0000820FEF7A7FE06210920FEF7A3FE062134
:103DC0000A20FEF79FFE06211720FEF79BFE062124
:103DD0002820BDE80840FEF795BE000008B5FFF7B3
:103DE00043FEFEF7B3FDFEF7A3FEFFF7A5F8FFF7CE
:103DF000FFFDBDE80840FFF7DBBC00001FB51C4617
:103E0000094B1B680546D86852B1084B02928DE8F1
:103E10000A0022462B460649FDF712FB00F042F845
:103E2000044B1A46F2E700BF142500207C45000829
:103E300089450008B73F000810B501390244904297
:103E400001D1002010BD10F8013B11F8014FA34231
:103E5000F5D0181B10BD00002DE9F8430746884631
:103E600091461E468BB10D46A8EB0500B54207EB07
:103E7000000402D20020BDE8F883324649462046BD
:103E8000FFF7DAFF18B1013DEEE7BDE8F883204601
:103E9000BDE8F883034611F8012B03F8012B002A33
:103EA000F9D1704708B5062000F02CF80120FFF783
:103EB00033FA00001F2938B504460D4604D91623ED
:103EC00003604FF0FF3038BD426C12B152F8213020
:103ED0004BB9204600F030F82A4601462046BDE89E
:103EE000384000F017B8012B0AD0591C03D1162313
:103EF0000360012038BD002442F825402846984739
:103F0000002038BD024B01461868FFF7D3BF00BF41
:103F10001425002038B5074C0023054608461146F5
:103F20002360FFF7FDF9431C02D1236803B12B6026
:103F300038BD00BFA8420020FFF7ECB940A2E4F171
:103F4000646891064E6F20617070207369670A0083
:103F5000426164206677206C656E67746820257501
:103F60000A0042616420626F6172645F69642025A7
:103F7000752073686F756C642062652025750A0072
:103F800042616420617070204352432030782530B4
:103F900038783A30782530387820307825303878BD
:103FA0003A3078253038780A00476F6F64206669A8
:103FB000726D776172650A00726563656976656422
:103FC0005F756E697175655F69645F6C656E203CD5
:103FD0002055415643414E5F50524F544F434F4C32
:103FE0005F44594E414D49435F4E4F44455F4944FC
:103FF0005F414C4C4F434154494F4E5F554E4951E0
:1040000055455F49445F4D41585F4C454E475448C4
:10401000002E2E2F2E2E2F546F6F6C732F41505F5A
:10402000426F6F746C6F616465722F63616E2E6393
:10403000707000616C6C6F63617465645F6E6F6457
:10404000655F6964203C3D20313237006F72672E16
:104050006172647570696C6F742E637561765F67E9
:1040600070730000766F69642068616E646C655FD0
:10407000616C6C6F636174696F6E5F726573706F92
:104080006E73652843616E617264496E7374616E0C
:1040900063652A2C2043616E6172645278547261A8
:1040A0006E736665722A290063616E617264496E7F
:1040B0006974000063616E6172645365744C6F6370
:1040C000616C4E6F646549440000000063616E617D
:1040D000726448616E646C6552784672616D650009
:1040E00063616E6172644465636F64655363616CA0
:1040F0006172000063616E617264456E636F646536
:104100005363616C61720000696E6372656D656E08
:10411000745472616E73666572494400656E7175A0
:1041200065756554784672616D6573007075736866
:104130005478517565756500707265706172654679
:104140006F724E6578745472616E736665720000AA
:10415000636F707942697441727261790000000086
:104160006465736361747465725472616E736665BD
:10417000725061796C6F6164000000006672656561
:10418000426C6F636B0000006269745F6C656E6700
:104190007468203E20300072656D61696E696E67DB
:1041A0005F62697473203E203000696E7075745FC1
:1041B0006269745F6F6666736574203E3D20626C51
:1041C0006F636B5F6269745F6F66667365740062CC
:1041D0006C6F636B5F656E645F6269745F6F666668
:1041E000736574203E20626C6F636B5F6269745FFD
:1041F0006F66667365740072656D61696E696E677E
:104200005F6269745F6C656E677468203C3D207204
:10421000656D61696E696E675F6269747300696E6E
:104220007075745F6269745F6F6666736574203C55
:104230003D207472616E736665722D3E7061796C9B
:104240006F61645F6C656E202A2038006F75747032
:1042500075745F6269745F6F6666736574203C3D58
:104260002036340072656D61696E696E675F6269E0
:10427000745F6C656E677468203D3D203000287265
:104280006573756C74203E20302920262620287204
:104290006573756C74203C3D203634292026262019
:1042A00028726573756C74203C3D206269745F6C84
:1042B000656E67746829000064657374696E617463
:1042C000696F6E20213D202828766F6964202A2995
:1042D00030290076616C756520213D202828766F95
:1042E0006964202A293029006F66667365745F77D8
:1042F000697468696E5F626C6F636B203C20283361
:104300003255202D205F5F6275696C74696E5F6F36
:1043100066667365746F66202843616E61726442DD
:104320007566666572426C6F636B2C2064617461A4
:10433000292900006F75745F696E7320213D202864
:1043400028766F6964202A29302900007372635F20
:104350006C656E203E203055000000002863616EC1
:104360005F696420262030783146464646464646F8
:104370005529203D3D2063616E5F696400000000A7
:10438000616C6C6F6361746F722D3E7374617469DC
:1043900073746963732E63757272656E745F75737F
:1043A0006167655F626C6F636B73203E2030000055
:1043B0007472616E736665725F696420213D2028A6
:1043C00028766F6964202A2930290000737461748B
:1043D000652D3E6275666665725F626C6F636B73B6
:1043E000203D3D202828766F6964202A2930290045
:1043F0002E2E2F2E2E2F6D6F64756C65732F6C69AA
:104400006263616E6172642F63616E6172642E63B8
:10441000006974656D2D3E6672616D652E64617410
:10442000615F6C656E203E203000000000000000DF
:10443000012F0008ED2E0008292F0008152F000875
:10444000212F00080D2F0008F92E0008E52E000886
:10445000352F000800400000004000000040000030
:104460000040000000000100000002000000020007
:10447000000002006D61696E0000000094440008B5
:10448000B0400020A842002001000000D9370008F9
:104490000000000069646C6500000000A0011028A5
:1044A00000000000AAAAAAAA50011000FFFF000005
:1044B000007700000000000000A40A0100000000D6
:1044C000AAA6AAAA80500000DFEF00000000007733
:1044D000880000000000000000000000AAAAAAAAAC
:1044E00000000000FFFF00000000000000000000CE
:1044F0000000000000000000AAAAAAAA0000000014
:10450000FFFF0000000000000000000000000000AD
:1045100000000000AAAAAAAA00000000FFFF0000F5
:10452000000000000000000000000000000000008B
:10453000AAAAAAAA00000000FFFF000000000000D5
:10454000000000000000000000000000AAAAAAAAC3
:1045500000000000FFFF000000000000000000005D
:1045600000000000000000000A0000000000000041
:104570000300000000000000000000002C20667511
:104580006E6374696F6E3A2000617373657274694B
:104590006F6E2022257322206661696C65643A2063
:1045A00066696C6520222573222C206C696E65205B
:1045B0002564257325730A0088BCFF7F0100000075
:1045C000FFFFFFFF6400000000000000FE2A010062
:1045D000D2040000182500200000000000000000A8
:1045E00000000000000000000000000000000000CB
:1045F00000000000000000000000000000000000BB
:1046000000000000000000000000000000000000AA
:10461000000000000000000000000000000000009A
:10462000000000000000000000000000000000008A
:08463000000000000000000082
:00000001FF
